:020000040000FA
:0600000000EF08F0120001
:0608000000EF08F01200F9
:06082A0001003410000083
:08083000000200003500000089
:08083800D9CFE6FFE1CFD9FFA3
:10084000040EE126DE6ADE6ADE6ADD6ADD52DD5212
:10085000FD0EDBCF00F0FE0EDBCF01F0026A036A73
:1008600001AE02D002680368D9CFE9FFDACFEAFF10
:10087000030EEB500318E8AE02D0033408D000504A
:10088000EE5C0150EE580250EE580350EE580FE265
:100890000C0EE66EE0EC07F0E552D9CFE9FFDACFB7
:1008A000EAFFEE2A000EEE22EE22EE22D1D7040E4F
:1008B000E15C02E2E16AE552E16EE552E7CFD9FF81
:1008C00012000F0EC16E070EB46E936A300E926E58
:1008D0000F0E946EF19E816A80901200D9CFE6FFD0
:1008E000E1CFD9FF020EE1268250020B01E0010E9A
:1008F000080DF3CF02F08250010B040DF3CF01F08D
:100900008050200B01E0010EE824006E8050100B97
:1009100001E0010E002401240224DE6EDD6ADECF38
:1009200000F0DDCF01F000C0F3FF01C0F4FF020EC4
:10093000E15C03E200D0E16AE552E16EE552E7CF07
:10094000D9FF12008092320EE66E0EEC08F0E552EE
:100950008084320EE66E0EEC08F0E5528094320E82
:10096000E66E0EEC08F0E55212008082320EE66E62
:100970000EEC08F0E5528084320EE66E0EEC08F0C4
:10098000E5528094320EE66E0EEC08F0E55212004D
:10099000380E816ED7DF320EE66EE66A4DDFE55225
:1009A000E552010E816ECEDF320EE66EE66A44DF5E
:1009B000E552E5520D0E816EC5DF320EE66EE66A37
:1009C0003BDFE552E552060E816EBCDF320EE66E6D
:1009D000E66A32DFE552E5521200010E816EB2DFA7
:1009E0000A0EE66EE66A28DFE552E5521200D9CF1C
:1009F000E6FFE1CFD9FF020E816EA4DF0A0EE66E9C
:100A0000E66A1ADFE552E552FD0EDBCFE6FFFE0E89
:100A1000DB50280DF350E552E724E76EFE0EE7CFDA
:100A2000DBFFFD0EDB6AFE0EDB50F36EFD0EDBCF4F
:100A3000F4FFF350F45C0BE2140E816E83DF320E90
:100A4000E66E0EEC08F0E552FD0EDB2AECD7E5521F
:100A5000E7CFD9FF1200D9CFE6FFE1CFD9FFFE0ED5
:100A6000DB50816E82DF320EE66E0EEC08F0E5524E
:100A7000E552E7CFD9FF1200D9CFE6FFE1CFD9FF8A
:100A8000FD0EDBCFE9FFFE0EDBCFEAFFEF500EE0FD
:100A9000FD0EDBCFE9FFDB2AFE0EDBCFEAFF01E331
:100AA000DB2AEF50E66ED7DFE552EAD7E552E7CF13
:100AB000D9FF12000001646B300E926EF00E936E3F
:100AC000EF0E606F60C081FF040E616F615100081E
:100AD00021E26051FE0BE842606F60C081FF050EAD
:100AE000E66EE66AA9DEE552E5528150100B09E098
:100AF0008150200B06E08150400B03E08150800BB9
:100B000001E10AD80001640502E1655104D06105E4
:100B1000616FDCD7CFD71200F00E936E81CF63F0F8
:100B200000016315626F0F0E6015606F60516211F6
:100B3000606F81CF63F0F00E6315626FF00E625D3F
:100B400001E0F7D7936A06D866C065F00001010E90
:100B5000646F12000001676B100E675D14E267514D
:100B6000EA6A000FE96E020EEA22EF50605D08E1CA
:100B70006751EA6A100FE96E020EEA22EFCF66F0C3
:100B80006729676FE9D766C081FF640EE66EE66A83
:100B900053DEE552E55212000001686B070E685DF6
:100BA0001DE288DF0001696F6851EA6A6A0FE96E29
:100BB000000EEA2269C0EFFF6851EA6A6A0FE96E27
:100BC000000EEA22EF50460802E108D004D069C0C6
:100BD000E6FF41DFE5520001682BE0D76851EA6A81
:100BE0006A0FE96E000EEA22EF6A12000001686BDC
:100BF000070E685D16E26851EA6A6A0FE96E000E38
:100C0000EA22EF50E66E27DFE55200016829EA6A22
:100C10006A0FE96E000EEA22EF5001E102D0682B64
:100C2000E7D71200D9CFE6FFE1CFD9FFE652F25065
:100C3000800B01E0010EDF6EF29EA69EA69CA684AC
:100C4000FE0EDB50A96EFD0EDB50A86E550EA76E92
:100C5000AA0EA76EA682A6B2FED7A694DF50E8B071
:100C6000F28EE8A0F29EE552E552E7CFD9FF1200DE
:100C7000D9CFE6FFE1CFD9FFA69CA69EFE0EDB50A2
:100C8000A96EA680A85000D0E552E7CFD9FF120088
:100C900018DE7EDE80A84BD0200EE66E020EE66ED9
:100CA000EBDEE552E552E66A010EE66EA0DEE552A5
:100CB000E55272DF0001776B786B040E78AF02D0DB
:100CC000D89003D0775D000E785915E26A0E77252B
:100CD000E96E000E7821EA6EEF50E66E2DC2E6FF57
:100CE000A1DFE552E55202012D2B000E2E2300015B
:100CF000772B7823E2D76A0EE66E000EE66E1CECC8
:100D000007F0E552E552F3CF73F0F4CF74F065DEEF
:100D1000250EE66E020EE66EAFDEE552E552E80EF7
:100D2000E66E030EE66E88DDE552E55243D0000123
:100D3000776B786B040E78AF02D0D89003D0775DD4
:100D4000000E785924E22DC2E6FF92DFE552E66EEE
:100D50006A0E00017725E96E000E7821EA6EE552F1
:100D6000E750EF6E02012D2B000E2E236A0E0001BC
:100D70007725E96E000E7821EA6EEF50E66E6BDEA5
:100D8000E55200016E6B772B000E7823D3D76A0EE5
:100D9000E66E000EE66E1CEC07F0E552E552F3CF6E
:100DA00073F0F4CF74F0E80EE66E030EE66E44DDE9
:100DB000E552E55212DE3E0EE66E4DDEE552ECDE09
:100DC0006A0EE66E000EE66E1CEC07F0E552E55288
:100DD000F3CF75F0F4CF76F000017351751902E18D
:100DE0007451761911E18080E80EE66E030EE66E0E
:100DF00023DDE552E5528090E80EE66E030EE66EC6
:100E00001BDDE552E55216D0E8DDE80EE66E030E76
:100E1000E66E12DDE552E5522F0EE66E020EE66E2C
:100E20002BDEE552E552E80EE66E030EE66E04DDBB
:080E3000E552E552BFD71200A4
:080E3800FF0EE3CFEAFFE552D3
:100E4000FF0EE3CFE9FFE552E66AE66AD9CFE6FF97
:100E5000DACFE6FFFC0EE124D96EFF0EE220DA6E57
:100E6000E66AE66AE66A200EEF5C06E0090EEF5CD1
:100E700003E0EF6603D03FD0EE50F5D72D0EEF5CC8
:100E800003E1FF0EE32A03D02B0EEF5C01E1EE50ED
:100E90002F0EEF6424D03A0EEF6021D0D890F90ED7
:100EA000E336FA0EE336FD0EDECFE3FFFE0EDDCFB6
:100EB000E3FFD890F90EE336FA0EE336D890F90E38
:100EC000E336FA0EE336FD0EE350DE26FE0EE35067
:100ED000DD22300EEE5CDE26000EDD22D9D7FF0EBD
:100EE000E3CFE8FFE85207E0F90EE31EE32AFA0E2B
:100EF000D8B4E306E31EE552E552E552FF0EE3CF18
:100F0000DAFFE552FF0EE3CFD9FFE552E1CFE9FF6B
:100F1000E2CFEAFFED52ED52EECFF3FFEFCFF4FF59
:020F20001200BD
:0E0F22002A0EF66E080EF76E000EF86E020133
:100F30000900F5503A6F0900F5503B6F03E13A673D
:100F400001D03DD00900F550356F0900F550366FDE
:100F50000900F550376F09000900F550E96E0900E6
:100F6000F550EA6E090009000900F550386F0900D4
:100F7000F550396F09000900F6CF3CF2F7CF3DF28A
:100F8000F8CF3EF235C2F6FF36C2F7FF37C2F8FFA0
:100F90000201385302E1395307E00900F550EE6EC3
:100FA0003807F8E23907F9D73CC2F6FF3DC2F7FF30
:100FB0003EC2F8FF02013A07000E3B5BBFD71200AA
:100FC000FF0EE350066E480E01D04C0EE76EE72E82
:100FD000FED7E76AE72EFED7062EF7D700001200ED
:100FE000000EF36E00EE00F0080E01D81200EA6069
:100FF00002D0EE6AFCD7F350E9601200EE6AFCD72B
:1010000012EE40F022EE40F0F86A059C91EC07F0F9
:0C10100019EC08F048EC06F0FBD71200C9
:04101C00FF0EE35090
:10102000E84E1200000000D000D000D0E82EFAD721
:021030001200AC
:021032001200AA
:0C103400EEEDEBE7DEDDDBD7BEBDBBB7A9
:101040007E7D7B7730313233343536373839414223
:1010500043444546636F646500636F6465206F6B4E
:09106000003C006572726F720021
:00000001FF
